:1000000088C00000A1C000009FC000009DC000008B
:100010009BC0000099C0000097C0000095C0000080
:1000200093C0000091C000008FC00000F9C3000021
:100030009CC4000089C0000087C0000085C000008B
:1000400083C0000081C000007FC000007DC00000B0
:100050007BC0000079C0000077C000006AC10000CA
:1000600073C0000071C000006FC000006DC00000D0
:100070006BC000002E034C005500460041002000DC
:100080005500530042002D0052005300320033004F
:1000900032002000410064006100700074006500BF
:1000A0007200000018034400650061006E0020002B
:1000B000430061006D0065007200610000000403F0
:1000C000090409023E00020100C0320904000001D7
:1000D0000202010005240010010424020605240682
:1000E0000001070582030800FF09040100020A005D
:1000F0000000070504021000050705830210000533
:100100001201100102000008EB034B200100010264
:10011000DC0111241FBECFEFD2E0DEBFCDBF11E066
:10012000A0E0B1E0E0EFFFE002C005900D92AC313D
:10013000B107D9F722E0ACE1B1E001C01D92A034D3
:10014000B207E1F75AD052C75BCF9BB1809590635D
:1001500089238BB90895FC01A081B1816C938081C2
:10016000918101969183808326813781821793073D
:1001700021F484819581918380832FB7F8948285BF
:1001800093850196938782872FBF0895FC01A281F2
:10019000B3818D91B383A28326813781A217B307E0
:1001A00021F424813581338322839FB7F8942285FB
:1001B000338521503109338722879FBF089584B743
:1001C000877F84BF0FB6F894A895809160008861FE
:1001D00080936000109260000FBE90E080E80FB640
:1001E000F89480936100909361000FBE8AB18063A0
:1001F0008AB98BB180638BB904C3E1DFE8E2F2E036
:100200004FB7F89488EA91E0918380839383828347
:100210009583848388E292E09783868320E830E0A8
:1002200031872087138612864FBFECE9F1E04FB784
:10023000F8948CE191E0918380839383828395830A
:1002400084838CE991E097838683318720871386A6
:1002500012864FBF80E279DF78948FB7F8942091AF
:100260003202309133028FBF80913002909131027F
:100270002817390749F080E091E0BAD597FD04C00E
:10028000682F88E292E067DF2FB7F8948091A6018B
:100290009091A7012FBF009729F48091C80085FD98
:1002A00021C032C0209101012F702093E9002091DC
:1002B000E80020FFF2CF8031910510F08FE090E050
:1002C000C82FE0919E01F0919F01608180E091E054
:1002D00027D5C1508111E1CF8CE991E057DFC111E1
:1002E000F0CFDBCF2FB7F894809132029091330298
:1002F0002FBF892B49F088E292E048DF9091C80037
:1003000095FFFCCF8093CE0080E091E05CD5CAD40D
:10031000A4CF80E11ACF80E218CF80E091E0DBD457
:10032000811102C080E201C080E10FCF80E091E046
:100330008CC51F920F920FB60F9211242F933F93EB
:100340004F935F936F937F938F939F93AF93BF93DD
:10035000EF93FF936091CE008EB3843089F48FB712
:10036000F8942091A6013091A7018FBF8091A4013C
:100370009091A5012817390719F08CE991E0EBDE7F
:10038000FF91EF91BF91AF919F918F917F916F916D
:100390005F914F913F912F910F900FBE0F901F9043
:1003A0001895CF93FC01818D813021F0823021F4AA
:1003B000C0E203C0C0E301C0C0E0808D823009F418
:1003C000C860828D873031F0883031F0863029F472
:1003D000C26003C0C46001C0C6605B9A1092C900CD
:1003E0001092C8001092CA0024893589468957891D
:1003F000DA01C901B695A79597958795BC01CD01FE
:10040000605C7D4B804F9F4FCFD521503109309399
:10041000CD002093CC00C093CA0082E08093C80036
:1004200088E98093C9005B98CF910895292F3327DD
:100430002230310559F02330310569F02130310582
:10044000F9F482E190E020E031E01EC08EE390E01C
:1004500022EC30E019C099278130910541F08230BB
:10046000910541F0892B61F4EEEBF0E005C0E4EA80
:10047000F0E002C0E4E7F0E0849190E09F0104C066
:1004800080E090E020E030E0FA013183208308959D
:1004900020913E0230913F022617370748F0611540
:1004A000710539F42091E8002E772093E80001C00F
:1004B000B90140E06115710579F12EB32223F1F104
:1004C0002530F1F12091E80023FD3CC02091E800A7
:1004D00022FD2EC02091E80020FFECCF2091F200F9
:1004E00030E0FC01CF016115710559F0283031056C
:1004F00040F481918093F100615071092F5F3F4F6B
:10050000F1CF41E02830310509F040E02091E800CA
:100510002E772093E800CECF4111CFCF09C08EB304
:10052000882361F0853061F08091E80083FD0AC086
:100530008091E80082FFF3CF80E0089582E0089583
:1005400083E0089581E0089520913E0230913F02BA
:100550002617370748F06115710539F42091E80036
:100560002E772093E80001C0B901FC0120E061155D
:10057000710561F18EB38823D9F18530D9F180916D
:10058000E80083FD39C08091E80082FD2BC0809196
:10059000E80080FFECCF8091F20090E061157105DA
:1005A00059F08830910540F424912093F100319660
:1005B000615071090196F2CF21E0089709F020E01F
:1005C0008091E8008E778093E800D1CF2111D2CFBF
:1005D00009C08EB3882361F0853061F08091E80016
:1005E00083FD0AC08091E80082FFF3CF80E0089588
:1005F00082E0089583E0089581E00895982F953072
:1006000058F59093E900981739F07091EC0020911B
:10061000ED005091F00003C0242F762F50E021FF11
:1006200019C03091EB003E7F3093EB003091ED002C
:100630003D7F3093ED003091EB0031603093EB0063
:100640007093EC002093ED005093F0002091EE00A9
:1006500027FF07C09F5FD3CF8F708093E90081E0B1
:10066000089580E00895EF92FF920F931F93CF9328
:10067000DF93E62EEC018C010C5F1F4FF12CFE1472
:1006800099F19881992359F1F801208169817A8142
:1006900031973081892F8F70853010F080E025C030
:1006A000223010F442E001C046E0E8E0F0E020E053
:1006B000E617F70720F42F5FEE0FFF1FF9CF229503
:1006C000207F422B232F2295220F220F207C991F5F
:1006D0009927991F622F692B91DF8823F9F2F394F0
:1006E00025960B5F1F4FCBCF81E0DF91CF911F91FC
:1006F0000F91FF90EF9008958091380287FF0FC00F
:100700008091E80082FD04C08EB38111F9CF10C042
:100710008091E8008B770AC08EB3882349F08091DE
:10072000E80080FFF9CF8091E8008E778093E800A1
:1007300008952091E4003091E50095E64091EC00A9
:10074000842F817040FF21C08091E80080FD1BC094
:100750008EB3882391F0853091F08091EB0085FD78
:1007600010C04091E4005091E5004217530731F367
:100770009A01915019F784E0089582E0089583E08A
:10078000089581E0089580E008954091E80042FFD7
:10079000DFCF08953FD041D08091D8008F778093EC
:1007A000D8008091D80080688093D8008091D800CC
:1007B0008F7D8093D80019BC82E089BD09B400FE0A
:1007C000FDCF1EBA109234021092360210923502FA
:1007D00042E060E080E012DF8091E1008E7F809354
:1007E000E1008091E20081608093E2008091E2006C
:1007F00088608093E2008091E0008E7F8093E0002B
:100800000895E3E6F0E080818E7F808381E080932D
:100810003702C0CF1092E20008951092E1000895CF
:100820001F920F920FB60F9211242F933F934F9365
:100830005F936F937F938F939F93AF93BF93EF9348
:10084000FF938091E10082FF0AC08091E20082FF65
:1008500006C08091E1008B7F8093E10022D28091DD
:10086000E10080FF16C08091E20080FF12C08091FD
:10087000E2008E7F8093E2008091E20080618093AD
:10088000E2008091D80080628093D80019BC1EBA23
:1008900042DD8091E10084FF2DC08091E20084FF61
:1008A00029C019BC82E089BD09B400FEFDCF80914A
:1008B000D8008F7D8093D8008091E1008F7E809357
:1008C000E1008091E2008F7E8093E2008091E2005F
:1008D00081608093E20080913402882311F084E0EB
:1008E00007C08091E30087FD02C081E001C083E082
:1008F0008EBB0FDD8091E10083FF26C08091E20076
:1009000083FF22C08091E100877F8093E10082E035
:100910008EBB109234028091E1008E7F8093E100C3
:100920008091E2008E7F8093E2008091E2008061FE
:100930008093E20042E060E080E060DE8091F000C1
:1009400088608093F000ADD1FF91EF91BF91AF919E
:100950009F918F917F916F915F914F913F912F91D7
:100960000F900FBE0F901F9018951F920F920FB609
:100970000F9211242F933F934F935F936F937F9325
:100980008F939F93AF93BF93CF93DF93EF93FF9397
:10099000C091E900CF708091EC00D82FD17080FD1C
:1009A000D0E81092E9008091F000877F8093F000FA
:1009B00078941ED01092E9008091F00088608093B6
:1009C000F000CD2BCF70C093E900FF91EF91DF9144
:1009D000CF91BF91AF919F918F917F916F915F91D7
:1009E0004F913F912F910F900FBE0F901F90189530
:1009F0001F93CF93DF93CDB7DEB7AA970FB6F894C6
:100A0000DEBF0FBECDBFE8E3F2E088E08E0F90912D
:100A1000F10091938E13FBCF89DC8091E80083FF76
:100A200028C18091380290913902953009F483C031
:100A300030F49130A9F168F0933091F11AC19830F7
:100A400009F4EDC0993009F4F9C0963009F011C1EC
:100A500093C0803821F0823809F00BC108C0809122
:100A6000350290913602992389F082600FC08091FF
:100A70003C028F70853008F0FCC08093E9008091C3
:100A8000EB0085FB882780F91092E9009091E8003F
:100A9000977F9093E8008093F1001092F100CAC014
:100AA000282F2D7F09F0E5C0882319F0823061F0EE
:100AB000E0C080913A02813009F0DBC0933009F048
:100AC00080E0809336022EC080913A0281112AC0C4
:100AD00080913C028F702FEF280F243008F0C9C09E
:100AE0008093E9002091EB0020FF1CC0933021F49B
:100AF0008091EB00806214C09091EB009061909324
:100B0000EB0021E030E0A90102C0440F551F8A9597
:100B1000E2F74093EA001092EA008091EB008860CF
:100B20008093EB001092E9008091E800877F80932A
:100B3000E800E2DD9EC081119CC010913A021F774F
:100B40008091E3008078812B8093E3008091E8001E
:100B5000877F8093E800D0DD8091E80080FFFCCFA4
:100B60008091E30080688093E300111102C082E06D
:100B700001C083E08EBB7DC08058823008F079C010
:100B800080913A0290913B028C3D53E0950771F5BC
:100B900083E08A838AE289834FB7F894DE01139653
:100BA00020E03EE051E2E32FF0E050935700E49163
:100BB00020FF03C0E295EF703F5FEF708E2F90E053
:100BC000EA3010F0C79601C0C0968D939D932F5FB9
:100BD000243149F74FBF8091E800877F8093E80078
:100BE0006AE270E0CE01019653DC13C060913C02D2
:100BF00070913D02AE014F5F5F4F18DCBC01892B45
:100C0000C1F19091E800977F9093E80089819A81E3
:100C10009BDC8091E8008B778093E8002AC08038C5
:100C200041F58091E800877F8093E800809134024D
:100C30008093F1008091E8008E7779CF811119C0FF
:100C400090913A029230A8F48091E800877F8093D7
:100C5000E8009093340250DD80913402811106C087
:100C60008091E30087FD02C081E001C084E08EBB7B
:100C700054DB8091E80083FF0AC08091E800877F01
:100C80008093E8008091EB0080628093EB00AA964D
:100C90000FB6F894DEBF0FBECDBFDF91CF911F918D
:100CA00008950895CF938EB3882399F0C091E900F9
:100CB000CF709091EC00892F817090FD80E8C82B57
:100CC0001092E9008091E80083FD92DECF70C0931E
:100CD000E900CF910895CF93DF93EC01FC0170966A
:100CE0008BE0DF011D928A95E9F782E08C8389878A
:100CF00083E08E8761E0CE010196B5DC882361F048
:100D000061E0CE010696AFDC882331F061E0CE01D0
:100D10000B96DF91CF91A7CC80E0DF91CF91089522
:100D20000F931F93CF932EB32430F9F4FC01048961
:100D3000158926893789012B022B032BB1F0C62F89
:100D400081818F708093E9008091E80085FF04C065
:100D5000C093F10080E00AC08091E8008E77809314
:100D6000E800E7DC8823A1F301C082E0CF911F9166
:100D70000F9108952EB3243021F5FC014489558943
:100D800066897789452B462B472BD9F081818F7057
:100D90008093E9008091F200882389F09091E80027
:100DA0008091E8008E778093E80095FD08C0C1DC53
:100DB000811108C08091E8008E778093E80080E080
:100DC000089582E008952EB3243089F4FC0144890B
:100DD000558966897789452B462B472B41F0218120
:100DE0002F702093E9002091E80020FDC3CF0895E3
:100DF0002EB3243019F08FEF9FEF0895FC01448942
:100E0000558966897789452B462B472BA1F3868127
:100E10008F708093E9008091E80082FFECCF809191
:100E2000F200882321F02091F10030E002C02FEF82
:100E30003FEF8091F200811105C08091E8008B772F
:100E40008093E800C90108950895CF93DF93EC01E2
:100E50008091E80083FFA5C0888190E020913C024A
:100E600030913D022817390709F09BC08091390263
:100E7000813261F020F4803209F43EC092C08232A7
:100E800009F46BC0833209F47CC08BC080913802B6
:100E9000813A09F086C08091E800877F8093E8005E
:100EA0008091E80080FFFCCF8C899D89AE89BF8945
:100EB0008093F100492F5A2F6B2F77274093F10031
:100EC000AD01662777274093F1008B2F9927AA273A
:100ED000BB278093F100888D8093F100898D8093EA
:100EE000F1008A8D8093F1008091E8008E778093E5
:100EF000E800DF91CF9100CC80913802813209F077
:100F000050C08091E800877F8093E8008091E800DE
:100F100082FD04C08EB38111F9CF43C03091F1003E
:100F20002091F1009091F1008091F1003C8B2D8B8C
:100F30009E8B8F8B8091F100888F8091F100898F3B
:100F40008091F1008A8F8091E8008B778093E80090
:100F5000D3DBCE01DF91CF9124CA80913802813258
:100F600001F58091E800877F8093E800C5DB8091E0
:100F70003A0290913B02998B888BCE01DF91CF9101
:100F800063CF80913802813261F48091E800877FDD
:100F90008093E800B1DB60913A02CE01DF91CF91FE
:100FA00053CFDF91CF910895A1E21A2EAA1BBB1B4C
:100FB000FD010DC0AA1FBB1FEE1FFF1FA217B30725
:100FC000E407F50720F0A21BB30BE40BF50B661F3B
:100FD000771F881F991F1A9469F7609570958095FF
:100FE00090959B01AC01BD01CF010895F894FFCF0E
:100FF00000831000000104100000018208000001BD
:0C100000000000000000000000000000E4
:00000001FF
